:100000000C942E010C944B010C944B010C944B015D
:100010000C944B010C944B010C944B010C944B0130
:100020000C944B010C944B010C94861C0C94581DA1
:100030000C9478170C944B010C944B010C944B01CD
:100040000C944B010C944B010C944B010C944B0100
:100050000C944B010C9400180C944B010C944B0124
:100060000C944B010C944B010C944B010C944B01E0
:100070000C944B010C944B010C944B010C944B01D0
:100080000C944B010C944B010C944B010C944B01C0
:100090000C944B010C944B010C944B010C944B01B0
:1000A0000C944B010C944B010C944B019803980356
:1000B000C403C4032C044A04620562055504EE041B
:1000C000FF04FF04C51DEC1DE41EEC1DE41E381EDC
:1000D0005B1EE41EB21EC11E1D011C0104000600B1
:1000E00007001600680069006A006B006C006D0074
:1000F0000A0336006B006500790000001603420019
:100100007200610074007A0077006F007200740062
:10011000680000000403090409023B00020100A07A
:10012000FA09040000010301010009211101000185
:1001300022400007058103080001090401000103B2
:1001400000000009211101000122B6000705820309
:100150002000011201000200000008EFBE070001AC
:10016000000102000105010902A10185020901A1A6
:100170000005091901290815002501950875018157
:10018000020501093009311581257F950275088125
:100190000609381581257F950175088106050C0A29
:1001A00038021581257F950175088106C0C00501BB
:1001B0000980A101850319012AB700150126B7009E
:1001C000950175108100C0050C0901A10185041974
:1001D000012AA002150126A002950175108100C018
:1001E00005010906A1018506050719E029E71500A3
:1001F00025019508750181020507190029EF1500F1
:10020000250195F07501810205081901290595055B
:1002100075019102950175039101C005010906A1BF
:1002200001050719E029E7150025019508750181E9
:10023000029501750881010507190029FF1500269F
:10024000FF00950675088100050819012905950527
:1002500075019102950175039101C00011241FBE23
:10026000CFEFDAE0DEBFCDBF11E0A0E0B1E0EEE21B
:10027000FFE302C005900D92A038B107D9F722E044
:10028000A0E8B1E001C01D92A237B207E1F70E94D9
:100290000B110C94951F0C940000811107C066236C
:1002A00011F081E001C080E00E94AA0181E0089580
:1002B00081E0089581E008950C945A0108950C940A
:1002C0005E011F93CF93DF9300D000D01F92CDB774
:1002D000DEB749835A836B833091830189819A8188
:1002E000311114C0662359F0222349F00E949F0760
:1002F000182F682F89819A810E94480703C00E94A5
:100300007307182F69817A81812F04C00E949F078B
:1003100069817A810F900F900F900F900F90DF916D
:10032000CF911F910C94C60EFC01262F4081518164
:100330006281738184810C94610181E00895CF937F
:10034000DF93EC0160E00E949401BE01DF91CF9148
:100350000C945F01CF92DF92EF92FF92C12CD12CCF
:100360007601C39404C0CC0CDD1CEE1CFF1C8A95E6
:10037000D2F78C2D0E943B0CC701B601FF90EF9085
:10038000DF90CF900C944A060C94F50F0C94F10F6B
:1003900008950E94F2050E94C8012FEF84E39CE0BB
:1003A000215080409040E1F700C000000C942618D6
:1003B0000F931F93CF93DF938C0161E00E94940110
:1003C000EC01B8010E945C018823F1F1B801CE0173
:1003D0000E94C2158823C1F1B801CE010E94A11369
:1003E000882391F1B801CE010E941E15882361F186
:1003F000F8018281882309F1CB358DE5D807C1F05A
:1004000050F4C115FCE5DF0781F0CF3DDC45A9F4D0
:100410000E94D50C19C0CC35EDE5DE0761F0CD3575
:10042000DD4559F40E94190C08C00E94C9010CC096
:100430000E94220C02C00E94250CC801DF91CF91BE
:100440001F910F910C94580180E0DF91CF911F9183
:100450000F9108950E9459170C9443020E9446027E
:100460000C945F1708950C94320281E008950C9467
:1004700035020895CF93C82F0E9433028C2F0E941B
:100480003702CF91089580E00C943A020E941E1624
:100490000C943A020E941E1690918201891721F055
:1004A000809382010C943A020895CF93DF93CDB7E5
:1004B000DEB72B970FB6F894DEBF0FBECDBF4F83CC
:1004C000588769877A878B8761110E94650B9E0127
:1004D0002F5F3F4F86E0F90111928A95E9F785E099
:1004E000FE013796D90101900D928A95E1F7898135
:1004F0009A814C815D81452B31F09F3F31F491E031
:100500008F3F19F403C091E001C090E090FF09C053
:1005100049815A816B817C818D819E810E94860AEE
:1005200005C0C9010E949D018111F2CF2B960FB623
:10053000F894DEBF0FBECDBFDF91CF910895FC01CF
:10054000808191810E94E1070895CF93882309F467
:1005500050C0C82F8CEF8C0F813AD0F46C2F809153
:100560000201909103010E949416882349F06C2F98
:1005700080910201909103010E941F170E94870B36
:100580006C2F80910201909103010E9414170CC0FE
:1005900080E28C0F883058F4C77081E001C0880F6A
:1005A000CA95EAF70E94480BCF910C94870BEBE5B4
:1005B000EC0FE33040F4F0E0E95BFE4F808190E027
:1005C000CF910C945216E8E5EC0FE73150F4F0E0CF
:1005D000EE0FFF1FE75EFE4F80819181CF910C945B
:1005E0006816CD3E30F08C2F0E949011CF910C9464
:1005F0006212CF910895882389F19CEF980F913A68
:1006000040F4682F80910201909103010E941F170E
:100610000DC090E2980F983058F4877091E001C0B7
:10062000990F8A95EAF7892F0E944E0B0C94870B3D
:100630009BE5980F933020F480E090E00C945216E4
:1006400098E5980F973120F480E090E00C946816BC
:100650008D3E20F00E94EB110C94621208951F93BE
:10066000CF93DF93182FEB010E94A502209741F052
:100670008FE99FE00197F1F700C000002197F6CFC6
:10068000812FDF91CF911F910C94FB02893319F0D8
:1006900060E070E002C060E570E00C942F038823F6
:1006A00021F00E94480B0C94870B0895882321F0B9
:1006B0000E944E0B0C94870B0895CF92DF92EF921D
:1006C000FF920F931F93CF93DF937C01D62FC72FF9
:1006D000FC011281058102950F700E943E0B882358
:1006E000B9F01123A9F08C2F807F803421F080E2B3
:1006F0008D0F883068F080915C0282FD09C082E035
:100700000E94E70B0E943E0B91E0D82ED92601C033
:10071000D12CCC2EC2948FE0C8228C2D90E08C304E
:10072000910508F0CFC1FC01EA5AFF4F0C942C1F31
:100730008C2F807FCF70882311F0C295C07F11234A
:1007400099F0CC2309F4AAC180E28D0F883010F013
:10075000D11104C08C2F0E94480B03C08C2F0E9423
:10076000580B0E94870B9AC18D2F0E94FB02CC234D
:1007700009F4A8C180E28D0F883038F1DD2329F11A
:100780008C2F0E945E0B24C08C2F807FCF70803214
:1007900011F0C295C07FDD2319F0D130A1F13DC029
:1007A00080915C0282FF17C0112349F0CC2329F00D
:1007B0008C2F0E94480B0E94870B80E070C180E064
:1007C0000E94FB02CC2309F47DC18C2F0E944E0BAA
:1007D0000E94870B77C1112371F0002341F0013093
:1007E00031F40E94680B8C2B0E94700B6BC10E942D
:1007F000680B8C2B1DC0002319F0013009F462C175
:100800000E947D0B25C0112321F0063008F05AC14B
:100810000EC0053008F056C11BC0112361F0002343
:1008200031F0F701858180FF39C18F7085838C2F6E
:100830000E944F0347C1002359F0D93309F03FC14B
:10084000FFEF07EE13E0F15000401040E1F735C133
:100850008C2F0E94560336C18C2F86958695837007
:1008600019F0813061F02EC1112321F08D2F9C2FC2
:10087000937002C080E090E00E9452162BC11123B9
:1008800021F08D2F9C2F937002C080E090E00E9499
:10089000681620C18D2F112319F00E94901102C0FB
:1008A0000E94EB110E94621215C18C2F837009F017
:1008B00047C011110BC12D2F229526952770220FAD
:1008C000220F6D2F6F70862F90E0A0E0B0E0022E17
:1008D00004C0880F991FAA1FBB1F0A94D2F7D4FF28
:1008E00010C04FE050E060E070E004C0440F551FBE
:1008F000661F771F2A95D2F74095509560957095A1
:1009000003C040E050E0BA01C695C695C3708A01A5
:100910009B01082B192B2A2B3B2BC901B801C23094
:1009200049F058F4C13019F00E945E06CFC00E9411
:100930004C06CCC00E947006C9C00E944A06C6C0C0
:10094000112319F08C2F817001C08695882309F43A
:10095000BDC02D2F229526952770220F220F6D2FB7
:100960006F70862F90E0A0E0B0E0022E04C0880FE8
:10097000991FAA1FBB1F0A94D2F7D4FF10C04FE0E3
:1009800050E060E070E004C0440F551F661F771F01
:100990002A95D2F7409550956095709503C040E038
:1009A00050E0BA01C695C695C3708A019B01082B19
:1009B000192B2A2B3B2BC901B801C23049F058F43E
:1009C000C13019F00E94230781C00E9411077EC028
:1009D0000E9435077BC00E94840678C0CF70112327
:1009E00039F08C2F0E94AA068D2F0E944F036EC0F3
:1009F0008D2F0E9456038C2F0E94CB0667C0D23FDA
:100A000021F128F4D03F41F0D13FC1F043C0D33FA2
:100A100019F1D43F79F03EC0112341F0053008F0C0
:100A200051C08C2F8F710E94F0064CC0063008F028
:100A300049C0F7CF80915C0282FF18C0112339F0C2
:100A40008C2F8F710E94AA063DC01123C9F38C2FF1
:100A50008F710E94CB0636C0112329F08C2F8F7125
:100A60000E9495062FC00E9490062CC0112349F0C9
:100A7000CF718C2F0E94AA0663E08C2F0E94CC0BB2
:100A800021C081E00E94E70B0230E0F082E00E948A
:100A9000E70B18C0112331F0002391F28D2F0E9433
:100AA000A50210C0002399F2D93349F41FEF27EEB5
:100AB00033E0115020403040E1F700C000008D2F9E
:100AC0000E94FB0288EF8C0D843020F40E941E16D9
:100AD0000E943A02DD20C9F00E943A0B80FD15C049
:100AE000F70112820E94340B0E94AA06C7010E94DD
:100AF000A6050E94340BDF91CF911F910F91FF90BB
:100B0000EF90DF90CF900C94CB06DF91CF911F91A7
:100B10000F91FF90EF90DF90CF9008950F931F9368
:100B2000CF93DF93EC01688179818A810E94EC0781
:100B30008C010E9447070E943806B801CE010E942E
:100B40005D03DF91CF911F910F910895CF93DF93B4
:100B5000EC01988189812B813C81232B31F08F3FDF
:100B600031F481E09F3F19F403C081E001C080E0CF
:100B700080FD1DC0CE010E94D801811110C00E94CD
:100B80003E0B8823A1F08A81882389F080915C0242
:100B900082FD0DC082E0DF91CF910C94E70BCE0176
:100BA0000E948E05CE01DF91CF910C949F01DF91C1
:100BB000CF91089580E090E00E94521680E090E08E
:100BC0000E9468160E94650B0E94870B0E94931377
:100BD0000C94621280910201909103010E942A17E5
:100BE0000C94DA050E94550B0C94EA0592959F70BF
:100BF000963079F010F4925001C09A50923068F417
:100C0000803F69F018F4883E40F409C0843F29F41D
:100C100006C0883E20F0813F11F080E0089581E019
:100C20000895FC01808191810E94E1070E94F605F0
:100C30000895CF93DF9300D000D01F92CDB7DEB7D9
:100C40000F900F900F900F900F90DF91CF9108951C
:100C5000CF93DF9300D000D000D0CDB7DEB726967B
:100C60000FB6F894DEBF0FBECDBFDF91CF910895D0
:100C7000089508950C9439060C943A060E943C0697
:100C800060938D0170938E0180938F0190939001FA
:100C90000C94DA050C943E060F931F9300918D017E
:100CA00010918E0120918F0130919001602B712B5A
:100CB000822B932B1F910F910C943E060F931F9341
:100CC00000918D0110918E0120918F013091900142
:100CD00060237123822393231F910F910C943E066E
:100CE0000F931F9300918D0110918E0120918F0120
:100CF0003091900160277127822793271F910F91D0
:100D00000C943E060C9439060E9482066093890179
:100D100070938A0180938B0190938C010C94DA0577
:100D200060E070E0CB010C9484060F931F9341E0C8
:100D300050E060E070E08A019B0104C0000F111FC9
:100D4000221F331F8A95D2F7C901B8011F910F9155
:100D50000C9484060F931F9341E050E060E070E034
:100D600004C0440F551F661F771F8A95D2F78091E4
:100D7000890190918A01A0918B01B0918C018A0127
:100D80009B01082B192B2A2B3B2BC901B8011F9162
:100D90000F910C9484060F931F9341E050E060E0A4
:100DA00070E004C0440F551F661F771F8A95D2F765
:100DB00040955095609570958091890190918A0138
:100DC000A0918B01B0918C018A019B01082319230A
:100DD0002A233B23C901B8011F910F910C9484066B
:100DE0000F931F9341E050E060E070E004C0440FB7
:100DF000551F661F771F8A95D2F7809189019091C0
:100E00008A01A0918B01B0918C018A019B01082776
:100E100019272A273B27C901B8011F910F910C946C
:100E200084060F931F930091890110918A012091EC
:100E30008B0130918C01602B712B822B932B1F9196
:100E40000F910C9484060F931F93009189011091C8
:100E50008A0120918B0130918C01602371238223C0
:100E600093231F910F910C9484060F931F9300916D
:100E7000890110918A0120918B0130918C016027AA
:100E80007127822793271F910F910C948406089550
:100E9000292F220F920F890FE82FE695E695E69508
:100EA000877051E001C0550F8A95EAF785E0E89F09
:100EB000F0011124EC57FE4F20E030E070E040815B
:100EC000CB01022E02C0969587950A94E2F78170B5
:100ED000819584278523842781932F5F3F4F253079
:100EE000310569F70895292F220F920F890F682F76
:100EF000669566956695982F977085E0689FB00116
:100F0000112440E050E080E0FB01E40FF51FEC57B6
:100F1000FE4F208130E0092E02C0369527950A94B5
:100F2000E2F721703327042E01C0220F0A94EAF75A
:100F3000822B4F5F5F4F4530510531F70895BF92C7
:100F4000CF92DF92EF92FF920F931F93CF93DF9395
:100F50008C01C0908901D0908A01E0908B01F090C3
:100F60008C0180918D0190918E01A0918F01B091A3
:100F70009001C82AD92AEA2AFB2ACFE1D0E0D7017A
:100F8000C6010C2E04C0B695A795979587950A942F
:100F9000D2F780FD04C0219790F7B12C07C0BC2E7A
:100FA000B8018C2F0E94DC0E0197A9F38B2DDF91E5
:100FB000CF911F910F91FF90EF90DF90CF90BF9056
:100FC0000895CF93DF93EC010E949F07BE010E941A
:100FD000DC0EDF91CF9108951F93CF93DF93EB0148
:100FE00090918301992321F0CB010E94E10713C066
:100FF000882349F0CB010E949F07182F682FCE014C
:101000000E94480704C0CB010E947307182FBE013D
:10101000812F0E94DC0EDF91CF911F9108951F93C5
:10102000CF93DF93C091910116E080919201C81790
:1010300099F0D0E01C9FF0011D9FF00D1124ED569A
:10104000FE4F4081518162817381848195810E942C
:1010500028062196C770E9CFDF91CF911F9108959F
:101060004091C3015091C4016091C5017091C601C6
:101070008091C7019091C8010C942806EF92FF92CD
:101080000F931F93CF93DF938091C80182958F7048
:1010900009F065C08091C501882309F460C0809182
:1010A0009101F09092011091C3010091C4016091EF
:1010B000C6017091C70191E01F3F09F090E0C09117
:1010C0000001D0910101292F96E0E92E8F1509F436
:1010D00046C06115710521F00F3F21F030E003C0DB
:1010E00031E001C0322F90E030FD36C0E89EF001C3
:1010F000E99EF00D1124DF01AD56BE4F11963C91D3
:101100001197301329C03C91311326C012963C919F
:101110001297311121C013964D915C911497461B83
:10112000570B4C175D07C0F48091C8018F70806128
:101130008093C801E856FE4F80818F708061808364
:1011400083EC91E00E94A605DF91CF911F910F9152
:10115000FF90EF900C940F0801968770B7CFDF9146
:10116000CF911F910F91FF90EF9008959F92AF92B2
:10117000BF92CF92DF92EF92FF920F931F93CF9384
:10118000DF93CDB7DEB761970FB6F894DEBF0FBE21
:10119000CDBF8C0185E0F801DE011D9601900D9216
:1011A0008A95E1F7D8011296EC909091C301E091F5
:1011B000C4012091C6013091C7012115310531F0DC
:1011C000EF3F31F481E09F3F19F403C081E001C09B
:1011D00080E0B82FB1709B2E80FD47C1D8014C91A3
:1011E00011965C9111971396AD90BC90149783EC77
:1011F000C82E81E0D82EF090C501B501621B730B9B
:101200002091000130910101FF2009F4D9C08091A3
:10121000C8016217730708F095C0282F207F09F0D6
:1012200052C05E1313C0491311C0FE2CE1100EC052
:101230008F7080618093C8010E943008C6010E94AF
:10124000A6058091C801F80185834DC1AB2831F016
:101250005F3F31F481E04F3F19F403C081E001C0EA
:1012600080E080FD03C081E08E2502C080E090E038
:10127000F82FF170FF2E80FF1CC08091910120910A
:10128000920136E0821709F40BC190E0389FF0011B
:10129000399FF00D1124ED56FE4F6181561306C0A3
:1012A0006081461303C06281E61203C00196877015
:1012B000E9CFFE2CEE2009F416C18091C8018160AF
:1012C0008093C80154C05E1306C0491304C0E110E6
:1012D00002C0F80199C0C8010E941106882361F17B
:1012E000EE2051F12091C801822F82958F7090E0FD
:1012F000029774F08091C3019091C40198878F8305
:101300001986BB86AA862C87CE0107960E94A60561
:1013100086E0F801A3ECB1E001900D928A95E1F727
:101320000E943E080E9430080AC05E1711F1C801F1
:101330000E94110681112CC0C8010E94A605FF243D
:10134000F394D1C0282F207F81F77A2DB98AA88AFB
:101350006E2D89890E94190683EC91E00E94A605F2
:1013600086E0D6011D928A95E9F70E943008F12C9B
:10137000BAC04913DCCFE110DACFF8018583C80188
:101380000E94A60586E0D6011D928A95E9F7ABC0BA
:10139000EE2091F22091C801822F82958F7090E00B
:1013A00002970CF4B5CF8091C3019091C4019A8348
:1013B00089831B82BD82AC822E83CE010196A6CF8B
:1013C0006217730708F044C0FE2CEE2009F4B4CF76
:1013D0005E1330C049132EC02091C80120FD21C0EA
:1013E000822F82958F70482F50E041155105C9F02A
:1013F000F80125834F30510541F08F5F982F92956A
:10140000907F822F8F70892B8583C8010E94A6054B
:1014100086E0F801A3ECB1E001900D928A95E1F726
:101420003CC086E0F801A3ECB1E001900D928A95F2
:10143000E1F759C0C8010E941106811169CF80915E
:10144000C80181608093C801C8010E94A6054BC0F5
:101450007A2DB98AA88A6E2D89890E94190686E09C
:10146000D6011D928A95E9F718C0EE2009F464CFE1
:10147000C8010E941106F82E882309F45DCF86E08A
:10148000F801A3ECB1E001900D928A95E1F783ECAD
:1014900091E00E949F020E943E080E94300823C0F3
:1014A0004D875E878D859E850E94E107292F2295B5
:1014B0002F70223028F49F7039F0811105C00BC0C5
:1014C000243028F49F7049F4805E883020F0C801F1
:1014D0000E94A6059F2CF92C06C0D80115969C9158
:1014E000907F91F7F8CF8F2D61960FB6F894DEBFFD
:1014F0000FBECDBFDF91CF911F910F91FF90EF9065
:10150000DF90CF90BF90AF909F9008951F93CF939F
:10151000DF93CDB7DEB72C970FB6F894DEBF0FBEC2
:10152000CDBF4F83588769877A878B879C87CE0189
:1015300007960E94B6088823D1F09F8188852A8566
:101540003B85232B31F08F3F31F481E09F3F19F42D
:1015500003C081E001C080E080FD47C04F81588515
:1015600069857A858B859C850E9428063EC086E029
:10157000FE013796DE01119601900D928A95E1F7F2
:10158000FF81E8856A857B856115710531F0EF3F44
:1015900031F481E0FF3F19F403C081E001C080E035
:1015A00080FD23C02091920130E0C901019687702F
:1015B00099274091910150E084179507F1F1F98343
:1015C000EA837D836C8396E0929FD001939FB00D58
:1015D0001124AD56BE4FFE01319601900D929A95A1
:1015E000E1F7809392010E940F0816E0809191012B
:1015F00090919201891771F1189FC00111248D56A5
:101600009E4F0E94B608882329F1E09191011E9F08
:10161000F0011124ED56FE4F4081518162817381AA
:10162000848195810E9428068091910190E0019625
:101630008770992780939101D9CF0E94F20510926B
:10164000920110929101E3ECF1E086E0DF011D923E
:101650008A95E9F72C960FB6F894DEBF0FBECDBF82
:10166000DF91CF911F9108958091E901859585952E
:10167000859508958091E901877008959091E90119
:10168000977081E009F480E0089580910C0208953C
:1016900090910C02892B80930C0208958095909173
:1016A0000C02892380930C02089510920C02089575
:1016B00090910B02892B80930B0208958095909155
:1016C0000B02892380930B02089510920B02089558
:1016D0008091EA01089508950C946B0B0C946C0BA7
:1016E00090915C0292FD08C09091EA01981721F058
:1016F0008093EA010C946E0B08958091EA0188238F
:1017000029F01092EA0180E00C946E0B0895CF93BB
:10171000DF93E0910201F091030180910C0280833C
:10172000E0910201F0910301908180910B02892BDD
:1017300080838091EA01882381F0E0910201F09199
:1017400003019081892B8083809102019091030194
:101750000E947E1681110E947D0BC0910201D091E2
:10176000030140E250E069EC71E0CE010E94461FA7
:10177000892B69F080E2FE01A9ECB1E001900D92A5
:101780008A95E1F7CE01DF91CF910C942A16DF9173
:10179000CF9108950C946B0B90915C0292FD10C058
:1017A00098E0899F90011124262B2093E9010E9443
:1017B000AA068091E9018595859585950C94CA0BBB
:1017C0000C94AA061092E90180E00C94CA0B2091B7
:1017D000E901809582238093E901982F977099F40D
:1017E00030E0482F082E000C550B2417350759F010
:1017F00090915C0292FD07C08595859585950E9424
:10180000CB060C94E20B089590915C0292FB222788
:1018100020F9281769F080FB92F990935C0280917F
:101820005B0290915C020E94510C82E00C94E70BE9
:10183000089580915C0282FB882780F991E08927D6
:101840000C94040C81E00C94040C80E00C94040CC7
:1018500080E090E00E945B1F21E0893E9E4F09F0EE
:1018600020E0822F089582E090E00C94531F83E0E3
:1018700090E00C94531F682F83E090E00C94611F5C
:10188000CF9384E090E00E94531FC82F82E290E043
:101890000E94531F2C2F30E0A901582BCA01CF9171
:1018A0000895CF93C92F682F84E090E00E94611FB4
:1018B0006C2F82E290E0CF910C94611FAB01BC01D0
:1018C0008FE090E00C94731FAB01BC0183E190E0CA
:1018D0000C94731F60E070E0CB010C94640C60E02A
:1018E00070E0CB010E945E0C0C946A0C69EE7EEFF6
:1018F00080E090E00E947F1F60E082E090E00E9424
:10190000611F60E083E090E00E94611F10928D01F2
:1019100010928E0110928F011092900160E084E08D
:1019200090E00E94611F60E082E290E00E94611FEF
:1019300060E085E090E00E94611F60E086E090E05A
:101940000E94611F6FEF87E090E00E94611F40E0FE
:1019500050E0BA0188E090E00E94731F60E08DE0E3
:1019600090E00E94611F40E050E0BA0188E190E001
:101970000E94731F60E087E190E00E94611F40E0D9
:1019800050E0BA018CE190E00E94731F60E070E0CB
:1019900080E290E00E947F1F40E050E0BA0188E1C1
:1019A00090E00E94731F0C946F0C0C94760C682FBF
:1019B0008EE090E00C94611F0E94E5176093130283
:1019C00070931402809315029093160260930F0295
:1019D000709310028093110290931202089585B7BC
:1019E000806885BF85B7806885BF089581E00895C8
:1019F0000C94F60C08950C94FA0C0C94FA0C0C94BC
:101A0000FD0C0C94FA0C0C94010D0C94FA0C0E9431
:101A1000EF0C88EB9FE00E9414160E94050D0C94B9
:101A2000030D0E94FB0C0C94FA0C0E94BB0F0C944B
:101A300039020E94D0170E9481100E94150D0E9449
:101A400019150C94FF0C8F929F92AF92BF92CF9278
:101A5000DF92EF92FF920F931F93CF93DF93CDB757
:101A6000DEB72A970FB6F894DEBF0FBECDBF0E9437
:101A70009010982E81110E94DC0C8DE0A82E82E03F
:101A8000B82E00E010E0802E802F0E94DF0FD82EAD
:101A9000F501C1905F01C826B1F40F5F1F4F0230FE
:101AA000110589F78FEF89838A831B820E94D917DA
:101AB0008160782F9D838C8349815A816B818D81D0
:101AC0000E9455022FC08091170281FD0E94E50FF0
:101AD000E12CFF24F3948C2D8F21F1F00E94F80C5F
:101AE000882399F0EE828F82DF2081E009F480E084
:101AF00088870E94D9178160782F9A8789874E81BD
:101B00005F8168858A850E945502F801E35FFD4F79
:101B10008081F826F08206C0E394FF0CF3E0EF1218
:101B2000DACFBBCF81E0911001C080E02A960FB6DA
:101B3000F894DEBF0FBECDBFDF91CF911F910F9103
:101B4000FF90EF90DF90CF90BF90AF909F908F90DD
:101B5000089580E00C94EF140E94230D0E94A90DBB
:101B60000E9480120C944A02CF93DF930E94E10EF0
:101B7000EC01811521E5920708F045C0811530E59B
:101B8000930708F094C0883E910528F5803E9105A2
:101B900008F0F8C0883A910570F4853A910508F08C
:101BA0007CC08130910509F475C008F4E8C0049741
:101BB00008F0E8C0E4C08F3B910508F0E0C0C85AC7
:101BC000D0E0CC0FDD1FC65BDE4F0990D881C02D61
:101BD000CE019464D8C0811540E2940758F4811571
:101BE00051E0950708F0CEC08D3E910508F4C7C0BE
:101BF0009065C9C0C11580E4D80708F4C0C0DF7083
:101C0000CE01906AC0C0811525E59207A8F4811520
:101C100034E5930708F095C0811543E5940708F073
:101C20007BC0811552E5950708F061C0D82FCC27FD
:101C3000CE01816F906AA7C0C11589E5D807A0F4CD
:101C4000C11528E5D20708F082C0C11536E5D307D3
:101C500008F095C08C2F0E94750F8F7190E0D82FDF
:101C6000CC27CE0190628FC0C1154AE5D40708F495
:101C700074C0CE0190568115904208F080C08D2F1F
:101C80008F710E94750FDD27D0628F71AE01582BC6
:101C9000CA0179C081E090E076C0C55AD0E0C8584A
:101CA000DE4F8881C82FD0E0CE0190646CC074E014
:101CB000969587957A95E1F7282F23703C2F3370FE
:101CC00081E090E002C0880F991F3A95E2F79C6886
:101CD000AC01522B9A019C2F9F709695969550E2DD
:101CE000959FE0011124C9018C2B9D2B4CC0837062
:101CF000992721E030E002C0220F331F8A95E2F7D6
:101D00009C2F9695969580E2989FE0011124C22B16
:101D1000D32BCE019C6837C08370992721E030E037
:101D200002C0220F331F8A95E2F79C2F9695969555
:101D300040E2949FE0011124C22BD32BCE019A687C
:101D400022C0D82FCC27CE01846F906A1CC0DC2F14
:101D5000CC27CE01806F906A16C08C2F8F700E94A6
:101D6000750F94E0D695C7959A95E1F7CF70D0E0BE
:101D7000DC2FCC27D0699E01282BC90104C080E04C
:101D800090E001C0CE01DF91CF910895272F30E080
:101D9000F901EE0FFF1F2E0F3F1FF90196E0899FFB
:101DA000E00DF11D1124E60FF11DEE0FFF1FE852AB
:101DB000FF4F8591949108950E94C60E0E94B40D24
:101DC00008958238910569F1B0F48133910509F4E1
:101DD0006DC048F48932910509F463C08A329105D7
:101DE00009F469C008958533910509F455C0893314
:101DF0009105B9F00895833E910569F138F4803E6C
:101E00009105B1F0823E910509F10895863E910554
:101E1000A9F1873E9105B9F1843E910509F064C0AE
:101E200023C020915B0220FD4FC021FD4DC00895CD
:101E300080915B0280FD44C080915C0280FF44C0C1
:101E400080915B0284FD42C083EE4DC080915B02B5
:101E500082FF38C0F5CF80915B0282FD33C0809154
:101E60005C0280FD31C0ECCF80915C0281FF32C00A
:101E700080915B0284FD2AC087EE35C080915B02B1
:101E800083FF26C0F5CF80915B0283FD21C0809146
:101E90005C0281FD1FC0ECCF80915B0285FD1CC000
:101EA0001DC080915B0285FD19C016C080915B0248
:101EB00086FD16C017C080915B0286FD13C010C05E
:101EC00089E311C082EE0FC080EE0DC080E00BC030
:101ED00086EE09C084EE07C089E205C085E303C031
:101EE0008AE201C081E390E0089590915B0292FF45
:101EF0000DC0282F2871283019F4877F846006C010
:101F0000282F2471243011F48B7F886093FF0DC03B
:101F1000282F2871283119F4877E846106C0282F64
:101F20002471243111F48B7E886120915C0220FFA2
:101F30000DC0382F3871383019F4877F816006C0A2
:101F4000382F3171313011F48E7F886021FF0DC040
:101F5000282F2871283119F4877E816106C0282F27
:101F60002171213111F48E7E886194FD877E089560
:101F700080E0089508950E94280C811102C00E94FB
:101F8000D50C0E94330C809317020E94400C909352
:101F90005C0280935B020E94BA0F0E94370C682F8C
:101FA00070E080E090E00E944A06609189017091A3
:101FB0008A0180918B0190918C010C948206E82F0C
:101FC000F0E0E15AFD4F80810895089580EA8A95F6
:101FD000F1F7089500C008950C94E60F08950C944D
:101FE000EE0F0C94EF0F0C94EE0F0C94F30FF8948B
:101FF000E82FE295EF70F0E031A1282F2F7081E0FB
:1020000090E001C0880F2A95EAF7982F90959323C6
:1020100091A392A1892B82A37894089584E30E94CE
:10202000F70F80E90E94F70F83E90E94F70F82E91A
:102030000E94F70F81E90C94F70FCF92DF92EF9295
:10204000FF920F931F93CF93DF938C01C62FD0E0A5
:10205000CE0182589E4F7C01FC0190819F3F09F484
:1020600047C0D62EF894E92FE295EF70F0E081A1F9
:102070009F7021E030E001C0220F9A95EAF7822B91
:1020800081A382A12095282322A378940E94EA0F9D
:10209000EBE7F1E04EE751E031E0C12C21912F3F19
:1020A00089F0A22FA295AF70B0E090968C9190E04D
:1020B0002F7002C0959587952A95E2F780FD02C0A2
:1020C000832F01C080E0C82A330F4E175F0731F716
:1020D000F70180818F3F11F00E94F70F61E0C1107E
:1020E00001C060E08D2D0E94EC0FC00FD11FC8828F
:1020F000DF91CF911F910F91FF90EF90DF90CF90E4
:1021000008950E940E101092600210925F021092C9
:102110005E0210925D0282E00E94C8100C94C4011D
:102120001F93CF93DF9300D0CDB7DEB71A82198209
:1021300060E0CE0101960E941D1061E0CE01019683
:102140000E941D1042E050E0BE016F5F7F4F8DE5A1
:1021500092E00E94461F11E0009709F410E0892BDD
:1021600031F089819A8190935E0280935D02212FE4
:1021700042E06FE572E08DE592E00E94C9100E9496
:10218000C601812F0F900F90DF91CF911F9108957D
:102190000895FF920F931F93CF93DF938C01F62E38
:1021A000D72FC42F222349F081E080931A020E9486
:1021B000D917909319028093180280911A028823EC
:1021C000C1F080911802909119020E94F1170597B1
:1021D00080F0EF2DFD2FD8014C2F50E0CD01801B5A
:1021E000910B841795071CF48D918193F7CF109272
:1021F0001A02DF91CF911F910F91FF9008950E94D5
:10220000DE190E94190D0C94EA190E94EE190E9421
:10221000AC0D0C94081A0E9477170E94C5190E94F1
:10222000070D0E94FF100E9405110E94110DFBCFA7
:102230008091210280FF06C06091090170E0660F65
:10224000771F26C081FF04C06091090184E005C0AA
:1022500082FF07C06091090188E0689FB0011124E6
:1022600017C0909120029923D1F060910801961730
:1022700088F72091090188E0289F90011124929FFE
:10228000A001939F500D112470E0CA010E94181FF5
:102290006038710540F46115710519F406C068E0F5
:1022A00070E0862F08958FE7089581E0089580916A
:1022B000210280FF08C06091050170E07595679567
:1022C0007595679521C081FF06C06091050170E09A
:1022D0007595679519C082FF04C06091050170E093
:1022E00010C090911F02992399F0609104019617F4
:1022F000A0F780910501899FC001112470E00E9420
:10230000181F6038710540F46115710519F406C095
:1023100061E070E0862F08958FE7089581E00895C9
:102320008D3E21F40E941811819504C08E3E29F43F
:102330000E9418118093250208958F3E21F40E9477
:102340001811819504C0803F29F40E9418118093D0
:1023500024020895893F19F40E94571105C08A3F4D
:1023600031F40E94571181958093260208958B3F86
:1023700021F40E945711819504C08C3F29F40E94DA
:1023800057118093270208959FE0980F983078F4B2
:1023900021E030E0A90102C0440F551F9A95E2F7F1
:1023A000CA0190912302892B8093230208958D3FC7
:1023B00021F48091210281600BC08E3F21F4809135
:1023C0002102826005C08F3F29F480912102846040
:1023D0008093210208958D3E39F49091250297FF54
:1023E00035C01092250259C08E3E29F490912502E5
:1023F0001916BCF32BC0909124028F3E29F497FF4D
:1024000025C01092240249C0803F19F41916CCF35C
:102410001DC090912602893F29F41916BCF4109230
:1024200026023BC08A3F19F497FF10C0F8CF8B3FBC
:1024300039F49091270297FF09C0109227022DC00E
:102440008C3F21F4909127021916BCF39FE0980F5E
:10245000983080F421E030E0A90102C0440F551FFC
:102460009A95E2F7CA01809590912302892380937F
:10247000230213C08D3F21F4809121028E7F0BC077
:102480008E3F21F4809121028D7F05C08F3F29F47A
:10249000809121028B7F80932102809124028111FF
:1024A00006C080912502811102C010922002809105
:1024B0002602811106C080912702811102C010926C
:1024C0001F0208950E94D91720912402211104C0EF
:1024D00020912502222321F090931E0280931D0259
:1024E00020912602211104C020912702222321F0ED
:1024F00090931C0280931B0282E292E00C9444169B
:10250000EF92FF920F931F93CF93DF9300D000D0F1
:1025100000D0CDB7DEB786E0E2E2F2E0DE01119650
:1025200001900D928A95E1F7E0902402F090250247
:102530000091260210912702109224021092250287
:102540001092260210922702E11003C0FF2009F426
:102550005DC080911D0290911E020E94F117AC0196
:1025600090912002992339F020910A0130E024173C
:10257000350758F04BC020910B018AE0289F90014D
:1025800011242417350718F041C09F3F19F09F5FB1
:1025900090932002EE2061F00E9418111E1414F096
:1025A0009FEF01C091E0989F902D112490932402F9
:1025B000FF2061F00E9418111F1414F09FEF01C05A
:1025C00091E0989F902D1124909325023091240240
:1025D0003323E1F0209125022223C1F045EB34039F
:1025E000C0011124992319F09093240203C081E0C3
:1025F0008093240235EB2303C0011124992319F0A1
:102600009093250203C081E080932502011103C04D
:10261000112309F45DC080911B0290911C020E945D
:10262000F117AC0190911F02992339F02091060116
:1026300030E02417350758F04BC0209107018AE09D
:10264000289F900111242417350718F041C09F3F9F
:1026500019F09F5F90931F02002361F00E945711B1
:10266000101614F09FEF01C091E0989F902D112457
:1026700090932602112361F00E945711111614F055
:102680009FEF01C091E0989F902D11249093270215
:10269000309126023323E1F0209127022223C1F05A
:1026A00045EB3403C0011124992319F090932602BD
:1026B00003C081E08093260235EB2303C00111247F
:1026C000992319F09093270203C081E08093270299
:1026D0008091240281110BC080912502811107C0D5
:1026E00080912602811103C08091270281110E94EE
:1026F0006212EB82FC820D831E8386E0FE0131961E
:10270000A2E2B2E001900D928A95E1F726960FB60B
:10271000F894DEBF0FBECDBFDF91CF911F910F9117
:10272000FF90EF900895E2E2F2E086E0DF011D9273
:102730008A95E9F71092200210921F02109221024E
:102740000895CF93DF93EC01FB018281882309F484
:102750003CC1C430FDE5DF0760F4CB3F9CE5D90701
:1027600088F49E0122503C452431310508F02EC1E9
:1027700009C0C236EDE5DE0729F0C63AFDE5DF0700
:1027800009F024C10E94400C90935C0280935B028C
:10279000C1318CE5D80709F4C6C008F042C0C93081
:1027A000ECE5DE0709F49BC000F5C5308CE5D807E1
:1027B00009F485C078F4C330ECE5DE0709F478C08D
:1027C00008F07AC0C230DC4509F0F5C080915B02A8
:1027D0008160EFC0C7309CE5D90709F478C008F0E4
:1027E0007AC080915B028061E4C0CD30FCE5DF07F8
:1027F00009F487C058F4CB309CE5D90709F479C0B7
:1028000008F07BC080915B0288606FC0CF30FCE530
:10281000DF0709F480C008F082C080915B02877FE7
:10282000C8C0CE3F9CE5D90709F471C000F5C53199
:10283000FCE5DF0709F485C068F4C3319CE5D907DE
:1028400009F475C008F095C00E94F20580915B0202
:102850008F77AFC0CC3FFCE5DF07A9F108F054C08B
:10286000CB3FDC4509F0A7C080915C0240C0C2307C
:10287000EDE5DE0709F489C058F4C1158DE5D807E8
:1028800009F45AC008F069C080915C0282602FC0D0
:10289000C236EDE5DE0709F47CC0C63AFDE5DF0788
:1028A00009F481C0C330DD4509F085C080E06EC009
:1028B00080915B0282607DC080915B0216C0809136
:1028C0005B02886076C080915C0282604FC080911C
:1028D0005B0280626EC080915B0280646AC00E946D
:1028E000F20580915B02806864C0846062C0816090
:1028F0003DC080915B028E7F5CC080915B028D7FCA
:1029000058C080915B0216C080915C0218C0809113
:102910005C028D7F2BC080915B028F7E4AC08091CC
:102920005B028F7D46C080915B028F7B42C08091AD
:102930005B02877F8B7F3DC080915C028D7F8E7FA5
:1029400015C080915B0282FB222720F991E092273B
:1029500090FB82F990FB83F92CC080915C02982F48
:10296000909591708E7F892B90FB81F980935C020A
:1029700022C00E94F20580915B0287FB222720F98A
:1029800091E0922790FB87F914C081E00E94D70C58
:1029900012C080915B0284FB222720F991E09227EC
:1029A00090FB84F906C080915B02982F909590FB74
:1029B00080F980935B0280915B0290915C020E949F
:1029C000510C0E94F20580E001C081E0DF91CF91BF
:1029D00008950C944D0181E008950C94EB14CF926E
:1029E000DF92EF92FF9296B196FBCC24C0F8D12CE7
:1029F000960191E02927622F617060932902690195
:102A0000330FEE08FF0890912802691302C0882353
:102A100059F080E00E94E914C701B6010E94ED144C
:102A20008091290280932802FF90EF90DF90CF9051
:102A300008953E98469A81E00C94EF14CF93DF936B
:102A400086319C4541F5EB010E94450B982F8A8108
:102A50002091020130910301882379F09A7A81E074
:102A600009F480E080932A02911102C069E201C05A
:102A700065E3C9010E9414170AC080912A028111DE
:102A800002C069E201C065E3C9010E941F170E94EC
:102A9000870B80E001C081E0DF91CF9108950F9313
:102AA0001F93CF93DF93C42FD22FFC018281882301
:102AB000C9F040932D020E94D91790932C02809365
:102AC0002B0280E28C0F883008F057C0C77081E07D
:102AD00001C0880FCA95EAF7DF91CF911F910F913E
:102AE0000C944F0380912D02481330C080912B022B
:102AF00090912C020E94F117883C910538F510E264
:102B00001D0FCD17B9F080E28C0F883040F4C770EC
:102B100081E001C0880FCA95EAF70E945603183079
:102B200028F581E09D2F977001C0880F9A95EAF7EC
:102B30000E944F03802F0E9446031830F0F4D77094
:102B400081E001C0880FDA95EAF70AC080E28C0FB5
:102B5000883098F4C77081E001C0880FCA95EAF701
:102B6000DF91CF911F910F910C945603802FDF912D
:102B7000CF911F910F910C944603DF91CF911F913C
:102B80000F9108950F939C01CB01243F4CE534072E
:102B900031F188F4293DFCE53F07D9F02A3D4CE5A9
:102BA000340779F1283D3C45A9F506E221EE41EED6
:102BB00068ED7CE52BC0263FFCE53F07E1F0A8F07F
:102BC000273F3C4539F507E225EE46EE67EF7CE509
:102BD0001DC007E225EE45EE69ED7CE517C006E273
:102BE00021EE40EE64EF7CE511C007E225EE44EEF5
:102BF00065EF7CE50BC006E221EE42EE66EF7CE578
:102C000005C008E221E045EE6AED7CE50E944F1523
:102C100080E008C0FC018281882319F010922D0207
:102C200001C081E00F91089590938101809380010C
:102C3000089590933302809332020895E091320216
:102C4000F0913302309721F00190F081E02D09944A
:102C500080E00895E0913202F0913302309799F0CC
:102C600020911801222359F020915B0227FF07C011
:102C7000DC012C9111962C93119726E02C93028065
:102C8000F381E02D09940895E0913202F09133022E
:102C9000309739F022E0DC012C930480F581E02D9F
:102CA0000994089520913002309131022817390794
:102CB00071F09093310280933002E0913202F091F2
:102CC0003302309721F00680F781E02D09940895B2
:102CD00020912E0230912F022817390771F090931E
:102CE0002F0280932E02E0913202F091330230974E
:102CF00021F00084F185E02D09940895FC013296BD
:102D000080911801882331F080915B0287FF02C017
:102D10009EE101C096E080E0915028F021912223AD
:102D2000D9F38F5FF9CF0895662351F120911801EF
:102D30002223E9F020915B0227FF19C0462F469518
:102D4000469546954E31E0F4677021E030E002C0D0
:102D5000220F331F6A95E2F7FC01E40FF11D828117
:102D600090E02823392381E0232B69F409C0FC017A
:102D7000329608962191621729F0E817F907D1F7E2
:102D800080E0089581E008959C01FC0132969FEF58
:102D900080E04191461789F09F3F19F4411101C02D
:102DA000982F8F5F8630A9F79F3F39F0F901E90F1F
:102DB000F11D97FDFA956283089508959C012A5F9D
:102DC0003F4FFC014281461301C0128201968217D7
:102DD0009307B9F70895262F2695269526952E3127
:102DE00068F4FC01E20FF11D677021E030E001C0E2
:102DF000220F6A95EAF78281282B22830895262FD5
:102E00002695269526952E3170F4FC01E20FF11DD2
:102E1000677021E030E001C0220F6A95EAF7209543
:102E2000828128232283089520911801222329F0EA
:102E300020915B0227FD0C94EB160C94C416209194
:102E40001801222329F020915B0227FD0C94FF1624
:102E50000C94DE1620911801FC013296222331F0E9
:102E600080915B0287FF02C08EE101C086E0DF0136
:102E70001D928A95E9F7089508950C943C1783E014
:102E8000809334020C943D17811102C081E001C08F
:102E900082E0809334020C943D170C94441781E037
:102EA000809334020C943D170C944F1708950C94A2
:102EB00056170C9457170C9456170C9456170C94DD
:102EC00056170E945D170E9490100E945B1780E0C9
:102ED0000E94DF0F811108C081E00E94DF0F91E0A6
:102EE000811103C090E001C091E0892F08950895F9
:102EF0001F920F920FB60F9211248F939F93AF934F
:102F0000BF9380913502811113C08091610290912D
:102F10006202A0916302B09164024196A11DB11DAD
:102F20008093610290936202A0936302B093640263
:102F3000BF91AF919F918F910F900FBE0F901F90F7
:102F4000189580916902843031F10E942A02109212
:102F5000350220E488E190E00FB6F894A8958093BC
:102F600060000FBE2093600083B7817F846083BFC1
:102F700083B7816083BF7894889583B78E7F83BF42
:102F80000FB6F894A89580916000886180936000E6
:102F9000109260000FBE08950E94F2050C942E025C
:102FA00082E084BD93E095BD9AEF97BD80936E005B
:102FB00008952FB7F8948091610290916202A091D8
:102FC0006302B09164022FBF08952FB7F894609107
:102FD00061027091620280916302909164022FBF3E
:102FE00008959C014FB7F89480916102909162021C
:102FF000A0916302B09164024FBF821B930B0895AE
:1030000078941F920F920FB60F9211248F939F9373
:10301000AF93BF938091610290916202A09163028D
:10302000B09164020196A11DB11D8093610290933D
:103030006202A0936302B0936402BF91AF919F912B
:103040008F910F900FBE0F901F90189587E797E70D
:1030500090930108809300089AE088E10FB6F894F5
:10306000A895809360000FBE90936000FFCF809181
:1030700059020895089522E02093E9002FEF30913E
:10308000E800215035FD06C035ED3A95F1F7000016
:103090002111F5CF2091E80025FF0BC040E050E062
:1030A00066E070E00E947A1A8091E8008E77809343
:1030B000E8000895CF93DF9320911801222339F07F
:1030C00020915B0227FF03C060E222E002C068E0BB
:1030D00021E02093E9002FEF3091E800215035FDE9
:1030E00006C035ED3A95F1F700002111F5CF20919A
:1030F000E80025FF1DC0EC0180911801811105C079
:1031000040E050E068E070E003C070E040E050E074
:10311000CE010E947A1A8091E8008E778093E800B1
:1031200080E2FE01A9E3B2E001900D928A95E1F7F9
:10313000DF91CF91089580933602709338026093A7
:10314000370280916902843001F582E08093E900C2
:103150008FEF9091E800815095FD06C095ED9A950E
:10316000F1F700008111F5CF8091E80085FF0DC0D7
:1031700040E050E063E070E086E392E00E947A1A5B
:103180008091E8008E778093E8000895BC0184E088
:103190000C949B18BC0183E00C949B1880916802EE
:1031A000811109C00E940B1C0E94681C8091E200E2
:1031B00084608093E20008951092680208950C9450
:1031C00054176091650281E0611101C080E00C94A8
:1031D0003F179091690281E0943009F080E060919E
:1031E00065020C94441742E061EC81E00E94841B6C
:1031F00042E261EC82E00E94841B9091690281E0CE
:10320000943009F080E0609165020C944D17809134
:103210006B02833009F461C030F4813071F0823088
:1032200009F49AC008958A3009F486C08B3009F4F5
:103230006CC0893009F0A8C020C080916A02813A30
:1032400009F0A2C08091E800877F8093E800809118
:103250006E0290916F02892B21F460E289E392E083
:1032600003C060E080E090E070E00E94C51A8091A9
:10327000E8008B778093E800089580916A0281329C
:1032800009F082C080916E0290916F02029708F05F
:103290007BC08091E800877F8093E8008091E80000
:1032A00082FD05C0809169028111F8CF6DC0209127
:1032B000F3008091F20090E0922B029731F480911C
:1032C000F100813011F0863021F48091F10080937B
:1032D00059028091E8008B7753C080916A02813A4D
:1032E00009F052C080916E0290916F02892B09F013
:1032F0004BC08091E800877F8093E8008091E800D0
:1033000080FFFCCF8091180136C080916A02813223
:10331000D9F580916E0290916F02892BA9F5809169
:10332000E800877F8093E8000E94B91B80916C02BF
:10333000809318010C94F20580916A02813221F584
:103340008091E800877F8093E8000E94B91B8091FC
:103350006D0280935A02089580916A02813AA1F425
:103360008091E800877F8093E8008091E80080FFEB
:10337000FCCF80915A028093F1008091E8008E7713
:103380008093E8000C94B91B089584B7877F84BFAD
:103390000FB6F894A89580916000886180936000D2
:1033A000109260000FBE90E080E80FB6F894809312
:1033B0006100909361000FBE0C944F170E940B1C8C
:1033C0000E94681CE2EEF0E0808184608083789443
:1033D0000C94FD1E8CE091E00C941916809169020A
:1033E0008530A9F480916902853079F40E94A11793
:1033F000809167028823B1F30E946117882391F3BB
:103400000E94641A0E94F205EDCF0C94CC17089527
:1034100008950C940B1A292F332723303105C9F056
:1034200060F42130310581F02230310509F044C0CB
:103430008BE390E028E131E043C021323105E1F037
:103440002232310549F138C082E190E023E531E0D4
:1034500037C099278130910549F028F0029761F52E
:10346000E0EFF0E005C0E4E1F1E002C0ECEFF0E0F5
:10347000849190E09F0124C06115710541F0613095
:103480007105D1F489E090E023E431E019C089E0CE
:1034900090E02AE231E014C06115710541F061301D
:1034A000710551F486EB90E025E631E009C080E437
:1034B00090E02BE132E004C080E090E020E030E0DA
:1034C000FA0131832083089580E189BD82E189BDBD
:1034D00009B400FEFDCF8091D8008F7D8093D80085
:1034E0008091E00082608093E0008091E00081FDA7
:1034F000FCCF0895CF92DF92EF92FF920F931F932C
:10350000CF93DF93EC018B017A010E94D81B8111CC
:1035100033C0E114F10439F0F70180819181081B77
:10352000190BC80FD91FC12CD12C0115110519F188
:103530008091E80085FD16C08091E8008E77809329
:10354000E800E114F10449F0F70180819181C80E8F
:10355000D91ED182C08285E00FC00E94D81B88236B
:1035600021F30AC089918093F10001501109FFEF06
:10357000CF1ADF0ADACF80E0DF91CF911F910F9150
:10358000FF90EF90DF90CF900895209170023091DE
:1035900071022617370748F06115710539F420913B
:1035A000E8002E772093E80001C0B901FC0120E07B
:1035B0006115710579F1809169028823F1F18530F7
:1035C000F1F18091E80083FD3CC08091E80082FD2C
:1035D0002EC08091E80080FFEBCF2091F300809116
:1035E000F20090E0922B6115710551F08830910541
:1035F00038F421912093F100615071090196F3CFC5
:1036000021E0089709F020E08091E8008E77809310
:10361000E800CECF2111CFCF0AC080916902882364
:1036200061F0853061F08091E80083FD0AC08091EF
:10363000E80082FFF2CF80E0089582E0089583E001
:10364000089581E00895209170023091710226174B
:10365000370748F06115710539F42091E8002E779D
:103660002093E80001C0B901FC0120E0611571055B
:1036700091F180916902882309F440C0853009F4F2
:103680003FC08091E80083FD3DC08091E80082FD4D
:103690002FC08091E80080FFE9CF2091F300809156
:1036A000F20090E0922B6115710559F08830910578
:1036B00040F424912093F1003196615071090196F4
:1036C000F2CF21E0089709F020E08091E8008E77A2
:1036D0008093E800CBCF2111CCCF0AC08091690242
:1036E000882361F0853061F08091E80083FD0AC095
:1036F0008091E80082FFF2CF80E0089582E0089593
:1037000083E0089581E00895982F973068F59093AD
:10371000E900981739F07091EC002091ED0050917C
:10372000F00003C0242F762F50E021FD02C09F5FE0
:10373000ECCF3091EB003E7F3093EB003091ED0009
:103740003D7F3093ED003091EB0031603093EB0022
:103750007093EC002093ED005093F0002091EE0068
:1037600027FDE5CF80E008958F708093E90081E028
:10377000089580916A0287FF11C08091E80082FD60
:1037800005C0809169028111F8CF11C08091E800D5
:103790008B770BC080916902882349F08091E80003
:1037A00080FFF8CF8091E8008E778093E80008953D
:1037B0002091E4003091E50095E64091EC00842FE3
:1037C000817040FF23C08091E80080FD1DC0809182
:1037D0006902882399F0853099F08091EB0085FD8E
:1037E00011C04091E4005091E5002417350729F3FA
:1037F000915011F09A01E1CF84E0089582E008959C
:1038000083E0089581E0089580E008954091E80004
:1038100042FFDDCF08950E94791C0E94811CE0EEDA
:10382000F0E0808181608083E8EDF0E080818F7737
:10383000808319BCA7EDB0E08C918E7F8C93808142
:103840008F7E80831092680208950F931F93CF9309
:10385000DF930E94791C0E94811CC8EDD0E0888112
:103860008F77888388818068888388818F7D88832B
:1038700019BC1092690210926502109267021092B0
:10388000660200EE10E0F80180818B7F80838881E2
:103890008160888342E060E080E00E94841BE1EE6A
:1038A000F0E080818E7F8083E2EEF0E080818160B5
:1038B0008083808188608083F80180818E7F80830F
:1038C000888180618883DF91CF911F910F91089546
:1038D000E8EDF0E080818F7E8083E7EDF0E080818D
:1038E0008160808384E082BF81E0809368020C94D1
:1038F000251CE8EDF0E080818E7F80831092E2004D
:1039000008951092DA001092E10008951F920F922C
:103910000FB60F9211242F933F934F935F936F93A2
:103920007F938F939F93AF93BF93EF93FF93809178
:10393000E10082FF0BC08091E20082FF07C080910E
:10394000E1008B7F8093E1000E94FC1E8091DA00F1
:1039500080FF1FC08091D80080FF1BC08091DA00DB
:103960008E7F8093DA008091D90080FF0DC080E1C6
:1039700089BD82E189BD09B400FEFDCF81E080935D
:1039800069020E94CE1805C019BC109269020E94FB
:10399000DC188091E10080FF19C08091E20080FF77
:1039A00015C08091E2008E7F8093E2008091E2005A
:1039B00080618093E2008091D80080628093D8007B
:1039C00019BC85E0809369020E94E1188091E100B2
:1039D00084FF30C08091E20084FF2CC080E189BD6B
:1039E00082E189BD09B400FEFDCF8091D8008F7DB2
:1039F0008093D8008091E1008F7E8093E1008091D8
:103A0000E2008F7E8093E2008091E20081608093EB
:103A1000E20080916502882311F084E007C0809164
:103A2000E30087FD02C081E001C083E0809369026A
:103A30000E94E9188091E10083FF29C08091E20093
:103A400083FF25C08091E100877F8093E10082E0C1
:103A500080936902109265028091E1008E7F8093CD
:103A6000E1008091E2008E7F8093E2008091E2008D
:103A700080618093E20042E060E080E00E94841B6D
:103A80008091F00088608093F0000E94DF18FF9121
:103A9000EF91BF91AF919F918F917F916F915F91C6
:103AA0004F913F912F910F900FBE0F901F9018953F
:103AB0001F920F920FB60F9211242F933F934F93A3
:103AC0005F936F937F938F939F93AF93BF93CF93A6
:103AD000DF93EF93FF93C091E900CF708091EC00EA
:103AE000D82FD17080FDD0E81092E9008091F000CD
:103AF000877F8093F00078940E949C1D1092E900CB
:103B00008091F00088608093F000CD2BCF70C0933F
:103B1000E900FF91EF91DF91CF91BF91AF919F911C
:103B20008F917F916F915F914F913F912F910F9066
:103B30000FBE0F901F9018951F93CF93DF93CDB7B3
:103B4000DEB7AA970FB6F894DEBF0FBECDBFEAE688
:103B5000F2E08091F100819322E0E237F207C9F7A9
:103B60000E9407198091E80083FF2EC180916A02AC
:103B700090916B02492F50E04A30510508F024C162
:103B8000FA01EE59FF4F0C942C1F803821F0823837
:103B900009F01AC108C080916602909167029923CA
:103BA00089F082600FC080916E028F70873008F0BC
:103BB0000BC18093E9008091EB0085FB882780F999
:103BC0001092E9009091E800977F9093E80080932D
:103BD000F1001092F100D1C0282F2D7F09F0F4C020
:103BE000882319F0823061F0EFC080916C0281303F
:103BF00009F0EAC0933009F080E0809367022EC09C
:103C000080916C0281112AC080916E028F702FEF1B
:103C1000280F263008F0D8C08093E9002091EB00EF
:103C200020FF1CC0933021F48091EB00806214C00F
:103C30009091EB0090619093EB0021E030E0A901BE
:103C400002C0440F551F8A95E2F74093EA00109294
:103C5000EA008091EB0088608093EB001092E9000D
:103C60008091E800877F8093E8000E94B91BACC078
:103C70008111AAC010916C021F778091E3008078B7
:103C8000812B8093E3008091E800877F8093E80098
:103C90000E94B91B8091E80080FFFCCF8091E30077
:103CA00080688093E300111102C082E001C083E0CC
:103CB0008093690289C08058823008F085C0809165
:103CC0006C0290916D028C3D53E0950779F583E08D
:103CD0008A838AE289834FB7F894DE01139620E045
:103CE0003EE051E2E32FF0E050935700E49120FFD3
:103CF00003C0E295EF703F5FEF708E2F90E0EA30E7
:103D000010F0C79601C0C0968D939D932F5F24310C
:103D100049F74FBF8091E800877F8093E8006AE20F
:103D200070E0CE0101960E94C51A16C060916E0225
:103D300070916F02AE014F5F5F4F0E94091ABC0184
:103D4000892B09F441C09091E800977F9093E80097
:103D500089819A810E94231B8091E8008B77809350
:103D6000E80032C0803881F58091E800877F809339
:103D7000E800809165028093F1008091E8008E77E1
:103D800072CF811121C080916C0290916D029927B0
:103D90000297D4F48091E800877F8093E8008091B7
:103DA0006C02809365020E94B91B809165028111AB
:103DB00006C08091E30087FD02C081E001C084E07D
:103DC000809369020E94F3188091E80083FF0AC083
:103DD0008091E800877F8093E8008091EB0080620B
:103DE0008093EB00AA960FB6F894DEBF0FBECDBF4E
:103DF000DF91CF911F9108950895CF93809169022B
:103E00008823A1F0C091E900CF709091EC00892F38
:103E1000817090FD80E8C82B1092E9008091E80045
:103E200083FD0E949C1DCF70C093E900CF9108953F
:103E300097FB072E16F4009407D077FD09D00E9457
:103E4000321F07FC05D03EF4909581959F4F089551
:103E5000709561957F4F0895EE0FFF1F0590F491C7
:103E6000E02D0994AA1BBB1B51E107C0AA1FBB1F71
:103E7000A617B70710F0A61BB70B881F991F5A95F6
:103E8000A9F780959095BC01CD010895FB01DC0157
:103E900004C08D910190801921F441505040C8F721
:103EA000881B990B0895F999FECF92BD81BDF89AB0
:103EB000992780B50895A8E1B0E042E050E00C9465
:103EC000871F262FF999FECF92BD81BDF89A0197E1
:103ED00000B4021639F01FBA20BD0FB6F894FA9A52
:103EE000F99A0FBE08950396272F0E94621F0E9421
:103EF000611F252F0E94621F242F0C94621F0196C0
:103F0000272F0E94621F0C94611FDC01CB01FC0172
:103F1000F999FECF06C0F2BDE1BDF89A319600B422
:0E3F20000D9241505040B8F70895F894FFCF2D
:103F2E00C800EB01280850011E0A140137185A1850
:103F3E003B18CA18C6183A1801E200E900EA00B5A3
:103F4E0000B600B700CD008301CC008A0192019427
:103F5E00012102230224022502260227022A02B38D
:103F6E0000B4006F007000818283E200E900EA0075
:103F7E00B500B600B700CD008301CC008A019201D6
:103F8E0094012102230224022502260227022A027C
:103F9E00B300B4006F0070008182839392913490CD
:00000001FF
